:020000040000FA
:1000000000000730990083169F01CD3085008113D1
:10001000831215141515A0019001FF3083169B0162
:10002000A120FF3083169B0AA12005168B10851690
:100030000230B32085120230B3208B1C1628051223
:100040002030051C1A30A1004E30051C4130A200A2
:100050007D2098200430A0077D2098200319412896
:10006000031841280430A007031837282C288316CA
:100070009B010301A12083169B0A0301A120051601
:10008000402883167C309B002608A12083169B0AFB
:100090002508A12083169B0A2408A12083169B0A09
:1000A0002308A120A509A609A50A0319A60A00008C
:1000B0002508A302031CA4032608A402A41B662887
:1000C000A00383167B309B000030A12083169B0188
:1000D0003430A120200883169B0AA12085168514A0
:1000E00078200000000000008510782000006F28B4
:1000F0001730FF3E031D792808002308A5002408B7
:10010000A60020088316900083120301013E031D00
:1001100086288E018F018B108B1C8C2810148B105D
:100120008B1C902810100E08A3000F08A4000800D4
:100130002108A302031CA4032208A4022408230408
:10014000080083169A001C1555309D00AA309D00AA
:100150009C1483128C1FAA288C130800A700B920B6
:10016000A70BAF280800A8006430AE20A80BB42865
:100170000800C6300000FF3E031DBA280000000042
:100180000000080043346F347034793472346934B9
:1001900067346834743420345034653474346534CE
:1001A00020344734723469346634663469347434C4
:1001B00068347334203428344334293420343234BE
:1001C00030343034373420343134323446343634F9
:1001D000323437342F3436343734353420344F34D6
:1001E00053344334433441344C3420347234653412
:1001F000633461346C34693462347234613474341D
:1002000069346F346E34203431342E343034333426
:02021000203498
:02400E00A43FCD
:00000001FF
